:1000000010308A00AD2800005034723465347634E4
:1000100072346134633465346E34FD3420347034AA
:1000200061346E3465346C3429340D340A34003450
:1000300050346F3464346134F83465346E34E934E8
:1000400020346E34613473347434613476346534FE
:100050006E34ED3420347634FD349A346B346134AC
:100060003A34203425344C3464340D340A340034AA
:1000700050346F3464346134F83465346E34E934A8
:1000800020346E34613473347434613476346534BE
:100090006E34ED34203461347A3469346D3475341F
:1000A00074343A34203425344C3464340D340A34F6
:1000B0000034D33C733AE5362037613AE131653795
:1000C0006910F030EE32EC3A20100D0500005A3481
:1000D0006134643461346E34E134203465346C341A
:1000E00065347634613463346534203425344C34DB
:1000F000643420340D340A3400345A3461346434A6
:1001000061346E34FD34203461347A3469346D34B2
:1001100075347434203425344C34643420340D3434
:100120000A3400344F08013A03199A28033A031994
:10013000A328AC2883168810831288108316081011
:1001400083120814B428831608108312081083162B
:10015000881083128814B42883168810831288109C
:10016000831608108312081008004F08013A03197B
:10017000BD28033A0319C628CF2883168811831295
:1001800088118316081183120815D72883160811C1
:10019000831208118316881183128815D7288316B5
:1001A0008811831288118316081183120811080020
:1001B0000830F80000008711A0112008831687007E
:1001C00000008312DD0D0712031CEC282016200806
:1001D00083168700F02883122012200883168700D8
:1001E00000008312A0152008831687008312871D44
:1001F000F728F80BDA2800008711A01120088316D1
:100200008700000083122016200883168700000054
:1002100000008312A0152008831687008312871D13
:100220000F29F8010000071A78148711A01120087F
:100230008316870083120712201220088316870076
:1002400083120800201620088316870000008312FE
:10025000A0152008831687000000831207122012C1
:10026000200883168700000083128711A011200840
:100270008316870038308312DD00D8202A30DD0055
:10028000D8200130DD00D8202012200883168700F6
:1002900000008312A0152008831687008312871D93
:1002A0004F290000532900002016200883168700DC
:1002B000000083128A110A1622294F30840083130A
:1002C0000008031970290230F800F701F70B6629BE
:1002D000F80B65299730F700F70B6C29800B632921
:1002E0000800201620088316870000008312A0153E
:1002F00020088316870000008312071220122008AE
:1003000083168700000083128711A011200883162E
:1003100087003C308312DD00D820DD01D820783002
:10032000DD00D820201220088316870000008312E9
:10033000A0152008831687008312871D9D290000C1
:10034000A12900002016200883168700000006302F
:100350008312CF005D21201620088316870000003D
:100360008312A0152008831687000000831207124D
:100370002012200883168700000083128711A01125
:100380002008831687003C308312DD00D82001301E
:10039000DD00D820DD01D820201220088316870038
:1003A00000008312A0152008831687008312871D82
:1003B000D7290000DB2900002016200883168700BB
:1003C000000006308312CF005D212016200883161E
:1003D000870000008312A015200883168700000004
:1003E0008312071220122008831687000000831250
:1003F0008711A0112008831687003C308312DD008E
:10040000D8200230DD00D820DD01D82020122008BD
:100410008316870000008312A0152008831687002A
:100420008312871D112A0000152A000020162008BB
:1004300083168700000006308312CF005D218A11E9
:100440000A162529A0132008831687008312871314
:100450000830F8002B2A0000F8173C2AF813D90CB2
:1004600003188717031C871378173C2A7813F80B97
:100470002F2A3A2A000087173F308400840B3E2A37
:100480000000F81B2E2A781B362A08008316031753
:100490008C170C140000000083120C087F3903191C
:1004A0008A2A0313C50003170D080313C600031798
:1004B0000F080313C7004508D90022224608031776
:1004C0008D000313470803178F0083168C170C1435
:1004D0000000000083120C0D0E0D7F3903198A2ACB
:1004E0000313C50003170D080313C60003170F08F5
:1004F0000313C7004508D9002222460803178D00C0
:100500000313470803178F008D0A03198F0A03137B
:10051000462A031703138A110A162E2920172008CA
:10052000831687008312071B932A0830F700C9013E
:10053000F717A82AF713A82A0310071B0314C90CDE
:100540007717A82A7713F70B9C2A4908F800B32AD3
:100550003F30F71B1130F800F80BAC2AF71B9A2A32
:10056000771BA22A9C2A0800F701F801480803100B
:100570004918F707F70CF80CC918F707F70CF80C2F
:100580004919F707F70CF80CC919F707F70CF80C1D
:10059000491AF707F70CF80CC91AF707F70CF80C0B
:1005A000491BF707F70CF80CC91BF707F70CF80CF9
:1005B00008001030CC00F701FA01C90CC80C031C6C
:1005C000E72A4A08F7070318FA0A4B08FA07FA0C51
:1005D000F70CF90CF80CCC0BDD2A08008316031776
:1005E0008C170C140000000083120D080313D000B8
:1005F00003170F080313D10003170C080313D900C6
:100600002222500803178D000313510803178F008F
:100610008D0A03198F0A0313CF0BEE2A0800D701A6
:100620000408D6005710831B5714D01F1F2BD61752
:10063000561ED60ACF09D009CF0A0319D00A500E88
:10064000F038D200D207E23ED300323ED500500847
:100650000F39D307D307D507E93ED400D407D40711
:100660004F0E0F39D407D507D40DD50DD509D50DAB
:100670004F080F39D507D20D0730D1000A30D50702
:10068000D403031C3F2BD407D303031C432BD307F2
:10069000D203031C472BD207D103031C4B2B513031
:1006A0008400831307305605561384035605031D33
:1006B000602B561A840A561A602B2030F7007D2BC7
:1006C000840755300402031956170008F700031D6C
:1006D000712B561B712B561A8B2BD619712B203070
:1006E0007C2BD61F792B2D30F70084035613D6139D
:1006F0007D2BD61556123030F707D0010408CF00F5
:100700005010831B50147708D90022224F08840010
:10071000831350188317840A561F612B0800083072
:10072000DE007708DF00201620088316870000000F
:100730008312A0152008831687008312871D9E2B25
:10074000071A0314071E0310F80D0000A01120085B
:100750008316870083128711DE0B932B2016200847
:10076000831687000000831207125F080319BD2B50
:10077000201220088316870083120000A01520088D
:10078000831687008312871DC32B00008711A011D9
:100790002008831687000000831207122012200809
:1007A0008316870083120800D901DA012016200879
:1007B0008316870000008312A01520088316870087
:1007C0000000831207122012200883168700000001
:1007D00083128711A01120088316870038308312F6
:1007E000DD00D8205708DD00D82020162008831609
:1007F000870000008312A0152008831687000000E0
:100800008312871D012C07122012200883168700EF
:10081000000083128711A011200883168700393049
:100820008312DD00D820F7018F237808DA00201228
:1008300020088316870000008312A0152008831665
:1008400087008312871D222C0000262C0000201612
:1008500020088316870000008312201620088316C4
:10086000870000008312A01520088316870000006F
:1008700083120712201220088316870000008312BB
:100880008711A01120088316870038308312DD00FD
:10089000D8205808DD00D8202016200883168700AD
:1008A00000008312A0152008831687000000831221
:1008B000871D582C0712201220088316870000007D
:1008C00083128711A0112008831687003930831204
:1008D000DD00D820F7018F237808D90020122008E6
:1008E0008316870000008312A01520088316870056
:1008F0008312871D792C00007D2C00002016200813
:100900008316870000008312DE015A08DD00DE0036
:10091000DD0159085D07F8005E08FA000318FA0ABD
:100920007808DB007A08DC005C08DE005B08DD008C
:10093000E0010430DF005E0860068039E200DE1F5F
:10094000A62CDD09DE09DD0A0319DE0AE01FAD2C45
:10095000DF09E009DF0A0319E00AF801F901F701EC
:10096000FA016008031DB72C5F080319D12C103061
:10097000E1000310DD0DDE0DF70DFA0D60087A02BF
:10098000031DC42C5F087702031CCD2C5F08F702FF
:10099000031CFA036008FA020314F80DF90DE10BC9
:1009A000B92CE21FD82CF809F909F80A0319F90A39
:1009B0007908DC007808DB005B08F8005C08F900C7
:1009C00008008E30F7005C08F8005B08F900FA01B7
:1009D000DC1FEF2CF809F909F90A0319F80AF808DD
:1009E000031DFC2C7908F800F9010830F702F8081B
:1009F000031DFC2CF701052D0310F81B032DF90D29
:100A0000F80DF703FC2CDC1FF81308006C08031921
:100A1000E02D8316A4007008031D102D8312E02D15
:100A2000A402031C1A2D7F30A407031C192D831266
:100A3000E02D242D8130A4020318202D8312E02DF7
:100A4000031D242D8312E02D2408F700F801F9017D
:100A5000FA01A30183126D088316A200A217831264
:100A60006E088316A10083126F088316A000193048
:100A7000A4007308A00203184D2D0130A102031831
:100A80004D2DA20203184D2DA30203184D2DA30ACC
:100A9000A20AA10A7308A0077F2D7208A1020318F9
:100AA000682D0130A2020318682DA3020318682DD7
:100AB000A30AA20A7208A1077308A007031C7F2DCE
:100AC000A10A031D7F2DA20A031D7F2DA30A7F2DDE
:100AD00071088038A20203187E2D0130A30203188A
:100AE0007E2DA30A71088038A2077208A107031C93
:100AF0005C2DA20A031D5C2DA30A5C2D7A14A40BA5
:100B0000822D8D2D0310A00DA10DA20DA30D03109C
:100B1000FA0DF90DF80DA50D392D251C952D031095
:100B2000F80CF90CFA0CA50C992DF70B992D8312E2
:100B3000E02DA51BC22D0310A00DA10DA20DA30D2C
:100B40007308A0020318AE2D0130A1020318AE2DC8
:100B5000A2020318AE2DA302031CD32D7208A1021A
:100B60000318B92D0130A2020318B92DA302031CEA
:100B7000D32D71088038A2020318C22D0130A302C0
:100B8000031CD32DFA0A031DD32DF90A031DD32DFF
:100B9000F80A031DD32DF70A031DD02D8312E02D73
:100BA000F80CF90CFA0C83126D088316A400710876
:100BB000A406A41FDD2DF817E52DF813E52D8312EB
:100BC000F701F801F901FA01831683120800690898
:100BD000F0006D08F006F01FF22D03110310E91B61
:100BE0000314252E6908F0006C08F1006808F10272
:100BF0000319002EF01F252E0308013A8300252E2D
:100C00006D08F1006908F10203190C2EF01F252E62
:100C10000308013A8300252E6E08F1006A08F102EC
:100C20000319182EF01F252E0308013A8300252EE4
:100C30006F08F1006B08F1020319242EF01F252E16
:100C40000308013A8300252E031008006C080319DD
:100C5000B22E8316A0007008031D302E8312B22E10
:100C6000A00703183E2E7F30A0020318392E8312EE
:100C7000B22E031D3D2E8312B22E442E8130A007CA
:100C8000031C442E8312B22E2008F700F801F9014C
:100C9000FA0183126D088316A400A41783126E084C
:100CA0008316A30083126F088316A2001830A000D9
:100CB000A101221C782E7308FA07031C652EF90A7D
:100CC000031D652EF80A0319A1177208F907031C02
:100CD0006C2EF80A0319A11771088312EE00EE17A3
:100CE0006E08F807031C772E8316A117831283164C
:100CF000A10DF80CF90CFA0CA40CA30CA20C031017
:100D0000A00B582E0130F707031C882E8312B22E39
:100D1000F81B922EA40DFA0DF90DF80DF70B922E7B
:100D20008312B22EA41FA52EFA0A031DA52EF90ABE
:100D3000031DA52EF80A031DA52EF80CF90CFA0CBC
:100D4000F70A031DA52E8312B22E83126D08831697
:100D5000A1007108A106A11FAF2EF817B72EF81336
:100D6000B72E8312F701F801F901FA0183168312F5
:100D700008008E30F7004F08F7025008F9005108BC
:100D8000F800F917F7080319D02E0310F908031D0E
:100D9000CC2EF8080319D02EF90CF80CF70BC52E41
:100DA000D01FD72EF809F909F80A0319F90A080023
:100DB0008A15DD238A117A08CA007908C9007808E3
:100DC000C8007708C7004A08D2004908D10048087F
:100DD000D0004708CF00B9267908CC007808CB00AE
:100DE0004B084502CF004608D0004C08031C4C0FAE
:100DF000D0025008CE004F08CD00CE08031D042FAE
:100E00004D08023C03184D2F4B084502031D0C2FC3
:100E10004C08460203194C2F4C084602031C1A2F9B
:100E2000031D162F45084B0203181A2F0230CF005E
:100E300092201D2F0130CF0092203230CF005D2153
:100E40000330CF0092203230CF005D218A15DD23A0
:100E50008A117A08CA007908C9007808C80077089A
:100E6000C7004A08D2004908D1004808D000470806
:100E7000CF00B9267908CC007808CB004B08450292
:100E8000CF004608D0004C08031C4C0FD00250087D
:100E9000CE004F08CD00042FFD2E0330CF0092204E
:100EA000183003178D0000308F001A300313CF0065
:100EB000EE22103084004C08D0004B08CF000F23E6
:100EC0000D30D90022220A30D90022228A110A16B6
:020ED000542AA2
:1010000080308318F1068316A201A30183126D08B4
:101010008316A1007108A10683126C080319042924
:101020008316A000F700700803190E29A002031907
:10103000A428031C5A287108A600A6177208A50048
:101040007308A400A3010310A60CA50CA40CA30C08
:10105000A00B2228A11F2F2822142829221020109B
:1010600022166F30840083133D292212A11B4228CF
:10107000201C4D28A60CA50CA40CA30CF70A0319E0
:1010800023294D28A61B50280310A30DA40DA50D40
:10109000A60DF7030319232942282217C628221375
:1010A00083126D088316A100A11F5828A6171C29BA
:1010B000A6131C297008A000F70083126C08831681
:1010C000A00283126D088316A600A61783126E086D
:1010D0008316A50083126F088316A400A3010310D2
:1010E000A60CA50CA40CA30CA00B6E28A11F7B289A
:1010F000A2142829A2102010A21673308400831392
:101100003D29A212A11B8E28201C9928A60CA50CF3
:10111000A40CA30CF70A031923299928A61B9C28C1
:101120000310A30DA40DA50DA60DF7030319232984
:101130008E28A217C628A2137108A100A11FA228F9
:10114000A6171C29A6131C297108A600A617720849
:10115000A5007308A400A11FB128A61322152829F1
:101160002211A30120106F30840083133D29A11B9D
:10117000DC2883126D088316A100201CC628A60C4B
:10118000A50CA40CA30CF70A03192329A31FD72825
:10119000A40A031DD728A50A031DD728A60A031DE4
:1011A000D728A60CA50CA40CF70A03192329221B87
:1011B0004F28A21B9B28FD288030A606A61FE428E6
:1011C00028297108A100F32883126D088316A10055
:1011D000A608031DF328A508031DF328A408031D72
:1011E000F328F7011C29A61BFD280310A30DA40D4D
:1011F000A50DA60DF70BF3282329A11F0129A6177A
:101200001C29A6131C2983127008F7007108831685
:10121000A6007208A5007308A4001C2983126C089C
:10122000F7006D088316A60083126E088316A500CA
:1012300083126F088316A4002608F8002508F90019
:101240002408FA005B29F701F801F901FA015B298A
:10125000A301A409A509A609A309A30A031D362908
:10126000A40A031D3629A50A0319A60A22182E2846
:10127000A2187A282219B028E1280008A407031C24
:101280004729A50A031D4729A60A03192014840328
:101290000008A507031C4F29A60A0319201484037C
:1012A0000008801F803AA60703182014221A352848
:1012B000A21A8128B728831208006710E7105A087D
:1012C000DE005908DD005808DC005708DB005A082A
:1012D000EB005908EA005808E9005708E800EF0158
:1012E000EE01ED01EC018A11E7258A15031C7C292A
:1012F00067145C08803ADC00EB01EA01E9017F3009
:10130000E8005E08EF005D08EE005C08ED005B0899
:10131000EC008A11E7258A15031CA729EF01EE01CD
:10132000ED017F30EC005E08F3005D08F2005C0820
:10133000F1005B08F0008A1106258A157A08DE00A4
:101340007908DD007808DC007708DB00E7140A3054
:10135000EF008930EE003430ED007C30EC005E08A8
:10136000F3005D08F2005C08F1005B08F0008A11F0
:1013700026268A157708E8007808E9007908EA0047
:101380007A08EB00EF007908EE007808ED007708A6
:10139000EC005E08F3005D08F2005C08F1005B08F9
:1013A000F0008A1126268A157708E8007808E900F7
:1013B0007908EA007A08EB0083107A08EF007908D0
:1013C000EE007808ED007708EC007C30F30079300F
:1013D000F2003530F1008130F00000207A08E200A0
:1013E0007908E1007808E0007708DF006208EF0084
:1013F0006108EE006008ED005F08EC005E08F30095
:101400005D08F2005C08F1005B08F0008A112626F6
:101410008A157708E8007808E9007908EA007A0870
:10142000EB00EF007908EE007808ED007708EC009B
:101430005E08F3005D08F2005C08F1005B08F00054
:101440008A1126268A157708E8007808E9007908C5
:10145000EA007A08EB0083107A08EF007908EE00C2
:101460007808ED007708EC003F30F3000230F2001E
:101470003330F1008330F00000207A08E200790870
:10148000E1007808E0007708DF006208EF006108FB
:10149000EE006008ED005F08EC005E08F3005D08F8
:1014A000F2005C08F1005B08F0008A1126268A151C
:1014B0007708E8007808E9007908EA007A08EB0084
:1014C000EF007908EE007808ED007708EC005E0880
:1014D000F3005D08F2005C08F1005B08F0008A117F
:1014E00026268A157708E8007808E9007908EA00D6
:1014F0007A08EB0083107A08EF007908EE0078088C
:10150000ED007708EC003330F3008C30F2001E3031
:10151000F1008330F00000207A08E2007908E10051
:101520007808E0007708DF00EF01EE01ED017F3081
:10153000EC005E08F3005D08F2005C08F1005B0857
:10154000F0008A1126268A157708E8007808E90055
:101550007908EA007A08EB00EF007908EE007808D5
:10156000ED007708EC005E08F3005D08F2005C080F
:10157000F1005B08F0008A1126268A157708E8003A
:101580007808E9007908EA007A08EB0083107A0805
:10159000EF007908EE007808ED007708EC001B30CA
:1015A000F300E430F2003530F1008230F00000202A
:1015B0007A08E6007908E5007808E4007708E30097
:1015C0006608EF006508EE006408ED006308EC00B3
:1015D0005E08F3005D08F2005C08F1005B08F000B3
:1015E0008A1126268A157708E8007808E900790824
:1015F000EA007A08EB00EF007908EE007808ED00C9
:101600007708EC005E08F3005D08F2005C08F1006A
:101610005B08F0008A1126268A157708E80078080A
:10162000E9007908EA007A08EB0083107A08EF00F5
:101630007908EE007808ED007708EC00A430F3009C
:10164000DB30F2006730F1008330F00000207A08D0
:10165000E6007908E5007808E4007708E30066080A
:10166000EF006508EE006408ED006308EC005E081A
:10167000F3005D08F2005C08F1005B08F0008A11DD
:1016800026268A157708E8007808E9007908EA0034
:101690007A08EB00EF007908EE007808ED00770893
:1016A000EC005E08F3005D08F2005C08F1005B08E6
:1016B000F0008A1126268A157708E8007808E900E4
:1016C0007908EA007A08EB0083107A08EF007908BD
:1016D000EE007808ED007708EC003330F3008C3032
:1016E000F2001E30F1008330F00000207A08E6009E
:1016F0007908E5007808E4007708E3005E08EF0069
:101700005D08EE005C08ED005B08EC006208F30089
:101710006108F2006008F1005F08F0008A112626D7
:101720008A157708E8007808E9007908EA007A085D
:10173000EB00EF007908EE007808ED007708EC0088
:101740006608F3006508F2006408F1006308F00021
:101750008A1106258A157A08E2007908E1007808DE
:10176000E0007708DF00E71CCF2B8314DB30EF00AD
:101770000F30EE004930ED007F30EC006208F300DE
:101780006108F2006008F1005F08F00000207A08AC
:10179000E2007908E1007808E0007708DF00671CC4
:1017A000D42B6008803AE0005F08F7006008F8007A
:1017B0006108F9006208FA0008000130D700023021
:1017C000D8008A11D4238A157908A8007808A700C0
:1017D0000330D7000430D8008A11D4238A15790841
:1017E000AA007808A9000530D7000630D8008A1171
:1017F000D4238A157908AC007808AB002808FA00D1
:101800002708A81F0C2C2708003CF700FA0128081D
:10181000031C280FFA027708AD007A08AE002A08E8
:10182000FA002908AA1F1D2C2908003CF700FA011C
:101830002A08031C2A0FFA027708D700FA30570744
:10184000AF007A08B0000318B00A2C08FA002B0881
:10185000AC1F332C2B08003CF700FA012C08031CAA
:101860002C0FFA027708D700FA305707B1007A0830
:10187000B2000318B20A2A08DC002908DB008A112A
:10188000E1248A157708D7007808D8007908D900AC
:101890007A08DA002C08DC002B08DB008A11E1242E
:1018A0008A155A08EF005908EE005808ED0057084D
:1018B000EC007A08F3007908F2007808F100770864
:1018C000F0008A1106258A157A08D2007908D1001D
:1018D0007808D0007708CF005208DA005108D90004
:1018E0005008D8004F08D7005D217A08D600790843
:1018F000D5007808D4007708D3005608EF005508C3
:10190000EE005408ED005308EC00C330F300F5304E
:10191000F2004830F1008030F0008A1106258A1567
:101920007708D7007808D8007908D9007A08DA0053
:10193000EF007908EE007808ED007708EC00F3017D
:10194000F2013430F1008630F0008A1126268A1523
:101950007A08D6007908D5007808D4007708D30033
:101960005308F7005408F8005508F9005608FA0023
:10197000F8135608D6005508D5007808D400530847
:10198000D300B01FC62CAE1FE32CC82CAE1BD22C2C
:1019900030082E02031CD22C031DE32C2D082F022D
:1019A000031CE32CB21FD72CAE1FE32CD92CAE1B8B
:1019B0000C2D32082E02031C0C2D031DE32C2D08C8
:1019C000310203180C2D043003178D0000308F00F6
:1019D00083168C170C140000000083128C08031966
:1019E0000A2D0D080313D70003170F080313D8009F
:1019F00003170C080313D9008A1122228A155708ED
:101A000003178D000313580803178F008D0A03195D
:101A10008F0AE82C982D0313AB08031D272DAC0863
:101A2000031D272DAA1B222DAA08031D1B2D2908E3
:101A3000003C0318222DD601D5013430D400863065
:101A4000D300262DD601D501D401D301972DAC1B8F
:101A5000642DAC08031D302D2B08003C0318642DA9
:101A6000AA1B4B2D8310EF01EE013430ED008530C1
:101A7000EC005608F3005508F2005408F100530832
:101A8000F00000207A08D6007908D5007808D40044
:101A90007708D300632D8314EF01EE013430ED009D
:101AA0008530EC005608F3005508F2005408F100A8
:101AB0005308F00000207A08D6007908D50078088D
:101AC000D4007708D300972DAA1B7F2D8314EF0134
:101AD000EE013430ED008630EC005608F300550876
:101AE000F2005408F1005308F00000207A08D600F4
:101AF0007908D5007808D4007708D300972D831093
:101B0000EF01EE010730ED008730EC005608F300DE
:101B10005508F2005408F1005308F00000207A083C
:101B2000D6007908D5007808D4007708D3000317C9
:101B30000313EB018030EA003130E9008730E80020
:101B40005608EF005508EE005408ED005308EC006D
:101B50008A11E7258A15031CB22DD601D501D401BF
:101B6000D301B22D5308F7005408F8005508F900C6
:101B70005608FA000800D901DA0120162008831659
:101B8000870000008312A01520088316870000003C
:101B90008312071220122008831687000000831288
:101BA0008711A0112008831687003C308312DD00C6
:101BB0008A11D8208A155708DD008A11D8208A1585
:101BC000201620088316870000008312A015200825
:101BD0008316870000008312871DEC2D0712201248
:101BE000200883168700000083128711A0112008A7
:101BF000831687003D308312DD008A11D8208A15B4
:101C0000F7018A118F238A157808DA00201220083C
:101C10008316870000008312A01520088316870012
:101C20008312871D112E0000152E0000201620089B
:101C30008316870000008312201620088316870071
:101C400000008312A015200883168700000083126D
:101C500007122012200883168700000083128711C4
:101C6000A0112008831687003C308312DD008A1102
:101C7000D8208A155808DD008A11D8208A15201628
:101C800020088316870000008312A0152008831601
:101C9000870000008312871D4B2E07122012200898
:101CA00083168700000083128711A0112008831675
:101CB00087003D308312DD008A11D8208A15F70194
:101CC0008A118F238A157808D900201220088316DC
:101CD000870000008312A015200883168700831256
:101CE000871D702E0000742E000020162008831619
:101CF000870000008312DE015A08DD00DE00DD01EE
:101D000059085D07DB005E08DC000318DC0A5B088D
:101D1000F8005C08F90008000330D7000430D80050
:101D2000BB257908A8007808A7000730D70008303D
:101D3000D800BB257908AA007808A9000530D7008B
:101D40000630D800BB257908AC007808AB0028081D
:101D5000FA002708A81FB52E2708003CF700FA0153
:101D60002808031C280FFA027708AD007A08AE0095
:101D70002A08FA002908AA1FC62E2908003CF700E5
:101D8000FA012A08031C2A0FFA027708AF007A0822
:101D9000B0002C08FA002B08AC1FD72E2B08003CF3
:101DA000F700FA012C08031C2C0FFA027708B10087
:101DB0007A08B2002A08DC002908DB008A11E12435
:101DC0008A157708D7007808D8007908D9007A08EA
:101DD000DA002808DC002708DB008A11E1248A15D4
:101DE0005A08EF005908EE005808ED005708EC00BB
:101DF0007A08F3007908F2007808F1007708F0001B
:101E00008A1106258A157A08D2007908D100780847
:101E1000D0007708CF005208DA005108D9005008E6
:101E2000D8004F08D7005D217A08D6007908D50080
:101E30007808D4007708D3005608EF005508EE0064
:101E40005408ED005308EC00C330F300F530F20005
:101E50004830F1008030F0008A1106258A15770895
:101E6000D7007808D8007908D9007A08DA00EF009E
:101E70007908EE007808ED007708EC00F301F20134
:101E80003430F1008630F0008A1126268A157A084F
:101E9000D6007908D5007808D4007708D300530815
:101EA000F7005408F8005508F9005608FA00F8132E
:101EB0005608D6005508D5007808D4005308D3003A
:101EC000A708031D7D2FA808031D7D2FAA1B762FB1
:101ED000AA08031D6F2F2908003C0318762FD6018E
:101EE000D5013430D4008530D3007C2FD601D50104
:101EF0000730D4008730D300D42FA81BA12FA80807
:101F0000031D862F2708003C0318A12FAA1FA02F0E
:101F10008314EF01EE013430ED008730EC005608F9
:101F2000F3005508F2005408F1005308F0000020B7
:101F30007A08D6007908D5007808D4007708D3004D
:101F4000D42FAA1BBC2F8314EF01EE013430ED0017
:101F50008630EC005608F3005508F2005408F100F2
:101F60005308F00000207A08D6007908D5007808D8
:101F7000D4007708D300D42F8310EF01EE01343062
:101F8000ED008630EC005608F3005508F2005408C6
:101F9000F1005308F00000207A08D6007908D50037
:101FA0007808D4007708D300EB018030EA003130A4
:101FB000E9008730E8005608EF005508EE005408A5
:101FC000ED005308EC008A11E7258A15031CED2F5C
:101FD000D601D501D401D301ED2F5308F7005408E1
:0C1FE000F8005508F9005608FA00080047
:102000000A128A158C260A168A117A08CA007908DB
:10201000C9007808C8007708C7004A08D2004908F4
:10202000D1004808D0004708CF000A12B9260A1686
:102030007908CC007808CB004B084502CF00460851
:10204000D0004C08031C4C0FD0025008CE004F08A3
:10205000CD00CE08031D30284D08023C0318872808
:102060004B084502031D38284C08460203198628F0
:102070004C084602031C4828031D422845084B0211
:10208000031848280230CF000A12B5200A164D283E
:102090000130CF000A12B5200A163230CF000A12E2
:1020A0005D210A160330CF000A12B5200A1632301D
:1020B000CF000A125D210A160A128A158C260A160A
:1020C0008A117A08CA007908C9007808C800770818
:1020D000C7004A08D2004908D1004808D000470884
:1020E000CF000A12B9260A167908CC007808CB006E
:1020F0004B084502CF004608D0004C08031C4C0F8B
:10210000D0025008CE004F08CD00302829280330D7
:10211000CF000A1292200A16383003178D000030C3
:102120008F001B300313CF000A12EE220A16103064
:1021300084004C08D0004B08CF000A120F230A1667
:102140000D30D9000A1222220A160A30D9000A12CA
:1021500022220A168A110A165A2A840183131F3072
:102160008305713083168F000F088312A013200897
:102170008316870083128717831603170908C0394F
:10218000890003131F129F12003003178800831267
:10219000870188018901FF300313A000A101A2017A
:1021A000831603170908C039890003131F129F12F1
:1021B000003003178800831203131F139F13831625
:1021C0009F1383121F149412A012200883168700F5
:1021D000831220162008831687008312A01120087E
:1021E0008316870001308312940000308316940018
:1021F0000108C73908388100831290010030F800C7
:102200009200003083169200831220152008831656
:1022100087008312970183169B019C0101309D006A
:102220008312031787018801890103300313CF004C
:102230000A1292200A160330CF000A12B5200A169D
:102240000A1222290A160A1271290A16593003178E
:102250008D0000308F000A120313462A0A16C301AC
:10226000C30A3730430784008313C8010408C7003A
:102270004810831B48140A128E220A16470884004D
:102280008313481883177808800037304307840089
:1022900083130008203C031D30290130C30243088A
:1022A000013A03195A29033A03195F29013A03191C
:1022B0007029992930303802B500B601992930309B
:1022C0003902C50030303802C700C8000A30C900E2
:1022D0000A12B4220A1678084507B500B6019929F2
:1022E00030303A02C50030303902C700C8000A3029
:1022F000C9000A12B4220A167808C507C7013808AF
:10230000C6003030C6020030031C0130C702470847
:10231000C9004608C800CB016430CA000A12D9229D
:102320000A1678084507B5007908B6000318B60AFA
:102330009929673003178D0000308F000F30031389
:10234000CF000A12EE220A16103084003608D000A0
:102350003508CF000A120F230A162030D9000A12BE
:1023600022220A160D30D9000A1222220A160A3039
:10237000D9000A1222220A16B801B701C201C1010E
:10238000C301C401C30A3730430784008313C80163
:102390000408C7004810831B48140A128E220A162C
:1023A0004708840083134818831778088000373063
:1023B0004307840083130008203C031DC229013019
:1023C000C3024308013A0319EC29033A0319F1291E
:1023D000013A0319022A2B2A30303802B300B40123
:1023E0002B2A30303902C50030303802C700C8000F
:1023F0000A30C9000A12B4220A1678084507B30049
:10240000B4012B2A30303A02C50030303902C700FF
:10241000C8000A30C9000A12B4220A167808C50793
:10242000C7013808C6003030C6020030031C013036
:10243000C7024708C9004608C800CB016430CA007B
:102440000A12D9220A1678084507B3007908B400A1
:102450000318B40A2B2A7D3003178D0000308F003B
:102460000E300313CF000A12EE220A161030840039
:102470003408D0003308CF000A120F230A16203088
:10248000D9000A1222220A160D30D9000A1222227D
:102490000A160A30D9000A1222220A163608C60085
:1024A0003508C5000A12D82E0A163408C6003308AB
:1024B000C50000280830C500FA30CF000A125D219F
:0A24C0000A16C50B5C2A2F296300E1
:04400E00F52CFF3F4F
:00000001FF
